:1000000017EF00F0EA6A050EE96EEF500EE00F0EF2
:10001000016E006A002EFED7012EFBD78F0E006EF8
:10002000002EFED70000EF2EF2D751EF00F0F86A55
:10003000D09EEA6AE96AC150C00B0F09C16E070E73
:10004000B46EC150C00B0F09C16EC090C092C09475
:10005000C09EC2809698C69A949E93809392010EF9
:10006000C66E000EC76ED190800ED56ECD6A000EA2
:10007000CA6E000ECB6EB16A9484BD6AB76AB66A66
:10008000070EB46E9250926E270E006E002EFED7B1
:1000900000D0B450A19CB56A040E956E320E056E68
:1000A000B1D78C988C9A8C9E83ACFED78C888C8E22
:0C00B0008C8A8C9A8C9E8C98F1D70300EF
:020000040030CA
:0E00000024CE390E0087A1000FC00FE00F4084
:00000001FF
